:10000000B1C4CBC4CAC420C5C8C4C7C4C6C4C5C44F
:10001000C4C4C4C4C2C46ECC97CCBFC4BEC4BDC427
:10002000BCC4BBC4BAC46ECA41C940C93FC93EC9F9
:100030003DC93CC93BC93AC939C969CA37C970CA3F
:1000400035C934C976CA78CA31C930C92FC92EC951
:100050002DC92CC92BC92AC929C928C971CA26C9C1
:1000600079CA24C923C922C921C920C91FC91EC9E7
:100070001DC91CC91BC91AC919C918C917C916C96C
:1000800015C914C913C912C911C910C90FC90EC99C
:100090000DC90CC90BC90AC909C908C907C906C9CC
:1000A00005C904C903C960CA01C900C9FFC8FEC89F
:1000B000FDC8FCC8FBC8FAC8F9C8F8C8F7C8F6C834
:1000C000F5C8F4C8F3C8F2C857CA58CAEFC8EEC892
:1000D000EDC85DCA7F7F8080818181828283838336
:1000E0008484848585868686878788888889898AA6
:1000F0008A8A8B8B8B8C8C8D8D8D8E8E8F8F8F9033
:1001000090919191929292939394949495959696BE
:100110009697979798989999999A9A9B9B9B9C9C4C
:100120009C9D9D9E9E9E9F9F9FA0A0A1A1A1A2A2DB
:10013000A3A3A3A4A4A4A5A5A6A6A6A7A7A7A8A869
:10014000A8A9A9AAAAAAABABABACACADADADAEAEFB
:10015000AEAFAFAFB0B0B1B1B1B2B2B2B3B3B3B48E
:10016000B4B4B5B5B6B6B6B7B7B7B8B8B8B9B9B923
:10017000BABABABBBBBBBCBCBCBDBDBEBEBEBFBFBA
:10018000BFC0C0C0C1C1C1C2C2C2C3C3C3C4C4C452
:10019000C5C5C5C6C6C6C6C7C7C7C8C8C8C9C9C9F0
:1001A000CACACACBCBCBCCCCCCCDCDCDCDCECECE8E
:1001B000CFCFCFD0D0D0D0D1D1D1D2D2D2D3D3D330
:1001C000D3D4D4D4D5D5D5D5D6D6D6D7D7D7D7D8D6
:1001D000D8D8D9D9D9D9DADADADBDBDBDBDCDCDC7D
:1001E000DCDDDDDDDDDEDEDEDFDFDFDFE0E0E0E029
:1001F000E1E1E1E1E2E2E2E2E3E3E3E3E4E4E4E4D7
:10020000E4E5E5E5E5E6E6E6E6E7E7E7E7E7E8E88B
:10021000E8E8E9E9E9E9E9EAEAEAEAEBEBEBEBEB42
:10022000ECECECECECEDEDEDEDEDEEEEEEEEEEEFFC
:10023000EFEFEFEFEFF0F0F0F0F0F1F1F1F1F1F1BD
:10024000F2F2F2F2F2F2F3F3F3F3F3F3F4F4F4F480
:10025000F4F4F4F5F5F5F5F5F5F6F6F6F6F6F6F64A
:10026000F7F7F7F7F7F7F7F7F8F8F8F8F8F8F8F816
:10027000F9F9F9F9F9F9F9F9F9FAFAFAFAFAFAFAE7
:10028000FAFAFAFBFBFBFBFBFBFBFBFBFBFBFCFCBF
:10029000FCFCFCFCFCFCFCFCFCFCFCFDFDFDFDFD99
:1002A000FDFDFDFDFDFDFDFDFDFDFDFDFEFEFEFE7A
:1002B000FEFEFEFEFEFEFEFEFEFEFEFEFEFEFEFE5E
:1002C000FEFEFEFEFEFEFEFEFEFEFEFEFEFEFEFE4E
:1002D000FEFEFEFEFFFEFEFEFEFEFEFEFEFEFEFE3D
:1002E000FEFEFEFEFEFEFEFEFEFEFEFEFEFEFEFE2E
:1002F000FEFEFEFEFEFEFEFEFEFEFEFEFEFDFDFD21
:10030000FDFDFDFDFDFDFDFDFDFDFDFDFDFDFCFC1F
:10031000FCFCFCFCFCFCFCFCFCFCFCFBFBFBFBFB22
:10032000FBFBFBFBFBFBFAFAFAFAFAFAFAFAFAFA27
:10033000F9F9F9F9F9F9F9F9F9F8F8F8F8F8F8F834
:10034000F8F7F7F7F7F7F7F7F7F6F6F6F6F6F6F643
:10035000F5F5F5F5F5F5F4F4F4F4F4F4F4F3F3F35A
:10036000F3F3F3F2F2F2F2F2F2F1F1F1F1F1F1F072
:10037000F0F0F0F0EFEFEFEFEFEFEEEEEEEEEEED90
:10038000EDEDEDEDECECECECECEBEBEBEBEBEAEAB2
:10039000EAEAE9E9E9E9E9E8E8E8E8E7E7E7E7E7D9
:1003A000E6E6E6E6E5E5E5E5E4E4E4E4E4E3E3E304
:1003B000E3E2E2E2E2E1E1E1E1E0E0E0E0DFDFDF31
:1003C000DFDEDEDEDDDDDDDDDCDCDCDCDBDBDBDB64
:1003D000DADADAD9D9D9D9D8D8D8D7D7D7D7D6D69B
:1003E000D6D5D5D5D5D4D4D4D3D3D3D3D2D2D2D1D4
:1003F000D1D1D0D0D0D0CFCFCFCECECECDCDCDCD10
:10040000CCCCCCCBCBCBCACACAC9C9C9C8C8C8C74F
:10041000C7C7C6C6C6C6C5C5C5C4C4C4C3C3C3C290
:10042000C2C2C1C1C1C0C0C0BFBFBFBEBEBEBDBDD4
:10043000BCBCBCBBBBBBBABABAB9B9B9B8B8B8B71F
:10044000B7B7B6B6B6B5B5B4B4B4B3B3B3B2B2B267
:10045000B1B1B1B0B0AFAFAFAEAEAEADADADACACB3
:10046000ABABABAAAAAAA9A9A8A8A8A7A7A7A6A602
:10047000A6A5A5A4A4A4A3A3A3A2A2A1A1A1A0A050
:100480009F9F9F9E9E9E9D9D9C9C9C9B9B9B9A9AA2
:1004900099999998989797979696969595949494F4
:1004A000939392929291919190908F8F8F8E8E8D47
:1004B0008D8D8C8C8B8B8B8A8A8A8989888888879A
:1004C00087868686858584848483838382828181EE
:1004D0008180807F7F7F7E7E7D7D7D7C7C7B7B7B42
:1004E0007A7A7A7979787878777776767675757496
:1004F0007474737373727271717170706F6F6F6EE9
:100500006E6D6D6D6C6C6C6B6B6A6A6A696968683C
:10051000686767676666656565646463636362628E
:100520006261616060605F5F5F5E5E5D5D5D5C5CDF
:100530005B5B5B5A5A5A5959585858575757565631
:10054000565555545454535353525251515150507F
:10055000504F4F4F4E4E4D4D4D4C4C4C4B4B4B4ACC
:100560004A4A494948484847474746464645454517
:1005700044444443434342424241414040403F3F60
:100580003F3E3E3E3D3D3D3C3C3C3B3B3B3A3A3AA8
:1005900039393938383838373737363636353535EA
:1005A000343434333333323232313131313030302C
:1005B0002F2F2F2E2E2E2E2D2D2D2C2C2C2B2B2B6A
:1005C0002B2A2A2A292929292828282727272726A4
:1005D00026262525252524242423232323222222DD
:1005E00022212121212020201F1F1F1F1E1E1E1E11
:1005F0001D1D1D1D1C1C1C1C1B1B1B1B1A1A1A1A43
:100600001A1919191918181818171717171716166D
:100610001616151515151514141414131313131396
:100620001212121212111111111110101010100FBC
:100630000F0F0F0F0F0E0E0E0E0E0D0D0D0D0D0DDB
:100640000C0C0C0C0C0C0B0B0B0B0B0B0A0A0A0AF8
:100650000A0A0A090909090909080808080808080E
:100660000707070707070707060606060606060622
:100670000505050505050505050404040404040431
:100680000404040303030303030303030303020239
:10069000020202020202020202020201010101013F
:1006A000010101010101010101010101000000003E
:1006B000000000000000000000000000000000003A
:1006C000000000000000000000000000000000002A
:1006D000000000000000000000000000000000001A
:1006E000000000000000000000000000000000000A
:1006F00000000000000000000000000000010101F7
:1007000001010101010101010101010101010202D7
:1007100002020202020202020202020303030303B4
:10072000030303030303040404040404040404048F
:100730000505050505050505050606060606060662
:100740000607070707070707070808080808080833
:100750000909090909090A0A0A0A0A0A0A0B0B0BFC
:100760000B0B0B0C0C0C0C0C0C0D0D0D0D0D0D0EC4
:100770000E0E0E0E0F0F0F0F0F0F10101010101186
:100780001111111112121212121313131313141444
:1007900014141515151515161616161717171717FD
:1007A00018181818191919191A1A1A1A1A1B1B1BB2
:1007B0001B1C1C1C1C1D1D1D1D1E1E1E1E1F1F1F65
:1007C0001F20202021212121222222222323232312
:1007D00024242425252525262626272727272828BB
:1007E00028292929292A2A2A2B2B2B2B2C2C2C2D62
:1007F0002D2D2E2E2E2E2F2F2F3030303131313106
:1008000032323233333334343435353536363637A5
:100810003737383838383939393A3A3A3B3B3B3C44
:100820003C3C3D3D3D3E3E3E3F3F3F4040404141E0
:100830004242424343434444444545454646464775
:10084000474748484849494A4A4A4B4B4B4C4C4C0D
:100850004D4D4D4E4E4F4F4F5050505151515252A1
:100860005353535454545555565656575757585832
:100870005859595A5A5A5B5B5B5C5C5D5D5D5E5EC4
:100880005F5F5F6060606161626262636363646452
:10089000656565666667676768686869696A6A6AE0
:1008A0006B6B6C6C6C6D6D6D6E6E6F6F6F7070716D
:1008B00071717272737373747474757576767677FA
:1008C0007778787879797A7A7A7B7B7B7C7C7D7D86
:1008D0007D7E7E7F33332E33330034352E3030002F
:1008E00037382E303000303830383039002F6D69CD
:1008F0006E000A417573736368616C743A004C61F1
:1009000075667A6569743A00487A0A506861736559
:100910003A2020004672657175656E7A3A002F6D37
:10092000696E20200A4973743A2000202020204458
:100930007265687A61686C202020200A20202020BF
:1009400000536F6C6C3A200053696E436F73200044
:100950002D2D2D2D2D2D2D2D2D2D2D2D2D2D2D2DC7
:100960000D0A000011241FBECFE5D4E0DEBFCDBFCD
:1009700010E0A0E6B0E0ECE3FDE102C005900D92CE
:10098000A636B107D9F710E0A6E6B0E001C01D9287
:10099000A93EB107E1F7D6D3D0C932CB1F920F924F
:1009A0000FB60F9211242F933F934F935F938F9322
:1009B0009F93AF93BF93EF93FF938091B200909179
:1009C000B300A091B400B091B5002091E200309145
:1009D000E3004091E4005091E500820F931FA41FB3
:1009E000B51F8093B2009093B300A093B400B0936E
:1009F000B500AD0156954795529542954F704527E4
:100A00005F70452724ED30E0FA01E20FF31FE49117
:100A1000E8BD8091BB009091BC00480F591F5770F2
:100A2000420F531FFA01A491AABDFF91EF91BF910C
:100A3000AF919F918F915F914F913F912F910F9027
:100A40000FBE0F901F9018951F920F920FB60F9226
:100A500011242F933F934F938F939F9345B14093CE
:100A6000BA0081E08093E6002091BD003091BE0085
:100A70002F5F3F4F8091B8009091B900009791F09F
:100A800001979093B9008093B800C09B04C08091F7
:100A9000E800481720F1C09B0DC08091B7008093FB
:100AA000E10032C08091E7008F5F8093E70089E921
:100AB00093E0E7CF8091B600841778F78091E1004A
:100AC000882399F4C09A8091AE009091AF00815034
:100AD00091F099279093AF008093AE0015C080915C
:100AE000E100882311F4C0980FC08091E10081508B
:100AF0008093E10009C0809166003093B10020939B
:100B0000B00020E030E0E5CF3093BE002093BD0080
:100B10009F918F914F913F912F910F900FBE0F900A
:100B20001F9018958A3028F4805D992787FD90954D
:100B30000895895C992787FD90950895AC01892BCC
:100B400061F020E030E0E6E6FEE0CF010197F1F74A
:100B50002F5F3F4F42175307C1F7089592B320E22A
:100B6000922792BB98B3977C98BB28B3982F969501
:100B700096959870292728BB28B3982F9695907240
:100B8000292728BB28B3982F96959695969590710E
:100B9000292728BB979892B3880F880F880F8078F1
:100BA000982792BB80E0982F9A95F1F795988A95AF
:100BB000F1F708951F93182FD1DF812F8295807F41
:100BC000CDDF1F9108951F93CF93DF93CFEBD0E03C
:100BD00010E40CC08A3019F0EDDF219607C096981A
:100BE00080ECE8DF82B3812782BB2196888188234D
:100BF00089F7DF91CF911F9108958EE190E09EDFFC
:100C0000969880E3ABDF8AE090E098DF80E3A6DF90
:100C100081E090E093DF80E3A1DF81E090E08EDF70
:100C200080E29CDF81E090E089DF88E2C3DF81E041
:100C300090E084DF81E090E081DF8CE0BBDF81E049
:100C4000B9DF82E090E07ADF82B390E4892782BB4B
:100C50000895969882E0AEDF82E090E06FDF82B385
:100C600090E4892782BB08959B01AC016115710551
:100C70008105910531F060E070E885EF90E213D8CE
:100C800004C020E030E040E050E0CA01B90108951E
:100C90002AE0660F771F881F991F2A95D1F72091A8
:100CA0006000309161004091620050916300FBD779
:100CB0009BE0220F331F441F551F9A95D1F72093B5
:100CC000E2003093E3004093E4005093E500089580
:100CD0000895823071F0833091F08130B1F0E0E01E
:100CE000F0E08FEF9FEF8F5F9740A8F0E0E0F2E039
:100CF00012C0AAE0B0E006D8CF010197F4CFA0E17E
:100D0000B0E000D8CF010197EECFA4E0B0E0FAD771
:100D1000CF010197E8CFCF01089588E081BDFFCFD3
:100D20001092E0000895EFEBF0E080E2819390E014
:100D3000E03EF907D9F71092680008951092680014
:100D40000895809168008150809368000895909183
:100D50006800EFEBF0E0E90FF11D8083892F8F5FD2
:100D600061E281D79093680008951F93182F88231C
:100D700021F080E2ECDF1150E1F71F9108951F93FD
:100D8000182F882321F080E3E2DF1150E1F71F9153
:100D90000895CF93DF93EC018881882329F0D7DF72
:100DA000219688818823D9F7DF91CF910895CF9339
:100DB000DF93FC018491882349F0EF012196C7DF7E
:100DC000FE012196E4918E2FEE23C9F7DF91CF919A
:100DD00008951F93CF93DF93EC01162F662369F0DC
:100DE000EFD590FDFDCF282F20532A3008F0275053
:100DF0002883115011F02196F3CFDF91CF911F91ED
:100E00000895CF93DF93CDB7DEB724970FB6F8944C
:100E1000DEBF0FBECDBF823039F1833041F181306A
:100E200049F1A0E0B0E019821A821B821C8284E0A2
:100E3000FE013196182E61D729813A814B815C8160
:100E4000DA01C90188589341A040B040895B994FAD
:100E5000A240B04090F020E533EC40E050E0298320
:100E60003A834B835C8309C0A6E0B0E0DCCFACE002
:100E7000B0E0D9CFA0E0B0E0D6CFCA01B901249646
:100E80000FB6F894DEBF0FBECDBFDF91CF910895AE
:100E9000CF93DF93CDB7DEB724970FB6F894DEBFBC
:100EA0000FBECDBF49835A836B837C83823049F068
:100EB000833061F0813079F0A0E0B0E040E050E0B4
:100EC0000EC0A6E0B0E04AE050E009C0ACE0B0E0FF
:100ED00040E150E004C0A0E0B0E044E050E084E035
:100EE000FE013196182E24D7DA0109011CD7249669
:100EF0000FB6F894DEBF0FBECDBFDF91CF9108953E
:100F00000F931F93CF93DF93CDB7DEB727970FB61D
:100F1000F894DEBF0FBECDBF4AE050E08E010F5FF8
:100F20001F4FB8012FD6C80178D527960FB6F89471
:100F3000DEBF0FBECDBFDF91CF911F910F910895FE
:100F40008DE059D58AE057D50895809164008823B3
:100F500039F080E599E06FD58FEB90E05ED5F0DF5A
:100F600078DE31DE08951F93182F82958F70DADDB9
:100F700042D5812F8F70D6DD3ED51F910895EF9217
:100F8000FF920F931F93CF93DF93CDB7DEB72497D4
:100F90000FB6F894DEBF0FBECDBF182F062F64E04A
:100FA000CE01019616DF8981E82EFF24E294F294A7
:100FB00050EFF522FE24E522FE248A81E80EF11C82
:100FC000E294F29440EFF422FE24E422FE248B818A
:100FD000E80EF11CE294F29430EFF322FE24E322B7
:100FE000FE248C81E80EF11C812FBDDF802FBBDF3A
:100FF0008091B600B8DF8091E800B5DF81E2FBD4D4
:101000008091E6008823E1F38091BA00F4D408943B
:10101000E108F108E114F10499F724960FB6F89469
:10102000DEBF0FBECDBFDF91CF911F910F91FF901B
:10103000EF900895CF93DF93CDB7DEB722970FB629
:10104000F894DEBF0FBECDBF62E0CE010196C1DED7
:10105000A981A295A07F8A81A80FBB27A050B0408C
:1010600044D6802D80DF22960FB6F894DEBF0FBEE7
:10107000CDBFDF91CF9108951F93CF93DF93CDB76D
:10108000DEB724970FB6F894DEBF0FBECDBF64E085
:10109000CE0101969EDE89818295807F9A81890F9B
:1010A0001B811295107F9C81190FA82FBB27A05080
:1010B000B040012E2CD657DF812F55DF24960FB676
:1010C000F894DEBF0FBECDBFDF91CF911F91089581
:1010D0000F931F938C01812F46DF802F44DF1F91D8
:1010E0000F91089587B38F6387BB80EF8FBD81E138
:1010F0008EBD8FEF90E097BD86BD89B7837C89BF99
:101100001ABC18BC81E083BF89B7816089BF8BE0BE
:1011100085BD89B7806889BF82E383BD87E090E0A1
:1011200038D487E886B980E687B9359A369A81B38C
:101130008C6F81BB82B38C6182BB85B38E6385BBB0
:101140005CDD08952F923F924F925F926F927F9253
:101150008F929F92AF92BF92CF92DF92EF92FF92C7
:101160000F931F93CF93DF93CDB7DEB7C554D04015
:101170000FB6F894DEBF0FBECDBFA7E1B0E0B5D586
:10118000902D84E6989FC0011124009709F0AFC309
:1011900028EE33E039AF28AFA4E1B0E0A6D5802D2A
:1011A000682EA2E1B0E0AED5FEABEDABFCE3F817E4
:1011B00018F466241EAA1DAAA5E1B0E0A3D5FCABD5
:1011C000EBABA8E1B0E09ED5F0936700E09366003A
:1011D000AAE1B0E08AD5802D1DA2813011F0F1E0A6
:1011E000FDA3AFE1B0E081D5802D99278093B700B2
:1011F000813110F01092B70080E1A0E2B0E09E01D2
:101200002F5F3F4F26963FAF2EAF2697F901182E3E
:1012100074D5798067DF84DD7894ABE1B0E065D583
:10122000802DA7E0DA2ED822ACE1B0E05ED5002D0B
:101230000770ADE1B0E059D5802DF7E0EF2EE82240
:1012400088E499E0B4DD86EE98E0B1DD7EDE10E062
:101250001FAA1AAA19AAFFEFF8AB1FA6882499247F
:101260005401222433242101E0E3FE2E1BA61CA6F8
:101270001DA61EA61AA619A62AE028A71FA21EA20E
:1012800088AD99ADAA27BB2724968CAF9DAFAEAF92
:10129000BFAF2497AD2DBB27BFAFAEAFE02FFF2769
:1012A000FDAFECAF2E2D33273BAF2AAF9C992DC15C
:1012B00002E09D9B03E083B3809586703EA13323BB
:1012C00009F067C1882319F08EA34AE04FA33AA919
:1012D000301769F0802F95DD1B012C01802FF9DC80
:1012E0009093BC008093BB000AAB4AE048A7809172
:1012F000E7005AA55817A1F18091E7008AA7821448
:101300009304A404B504E1F082149304A404B50486
:1013100008F0ABC124968CAD9DADAEADBFAD2497AA
:10132000880D991DAA1DBB1D52014101821593050F
:10133000A405B50510F44C015D01C501B401A8DC9C
:101340006091B0007091B100882799278DDC6BA760
:101350007CA78DA79EA73FA1332311F031503FA357
:101360004DA1442381F48091E600882361F08091AF
:10137000BA0058A9851708F0EEC19FA5992309F472
:101380008CC291509FA78091E7008A3008F478C002
:101390008091E7008A508093E7004FA94F5F4FABE1
:1013A00058A5552309F48FC1515058A74F2D4160BE
:1013B0008BA99CA9009709F407C101979CAB8BAB43
:1013C000892B09F001C14F7671E09AA9923009F496
:1013D00000C1933009F401C282E0F0E8FF2EF40E60
:1013E000A1EFFA22F8264F2D552782B3837E82BBC8
:1013F00062B39A010EAC02C0359527950A94E2F7C4
:1014000021703070220F331F220F331FCA010CAC22
:1014100002C0959587950A94E2F781709070880FC5
:10142000991F880F991F880F991F282B0AAC02C09B
:10143000559547950A94E2F7417050704295529540
:10144000507F5427407F5427242B262722BB772305
:1014500009F05EC17ADD7A9469F012C010E0E0E034
:10146000F0E021E030E02C0F3D1FE20FF31F708011
:10147000772031F41F5F133088F7E12FFF27F1CF7A
:101480003FA93C33B0F03C533FAB6394862D65E0FD
:10149000EAD3992351F4A2E1B0E04DA95EA90A0173
:1014A00042D4A4E1B0E0062C32D459A5552309F06A
:1014B00048C18BE3861538F494EC690EADA9BEA93A
:1014C0001196BEABADAB2FDCC090BB00D090BC0082
:1014D000113009F49AC0113008F47DC0123009F4BB
:1014E0007EC16ED290FDE2CE992787FD9095A92FFF
:1014F000B92FFC01B197E735F10508F0D7CEED5EC5
:10150000FF4F09940ADC9C9BD3CE01E0D2CE8AE047
:1015100090E0A0E0B0E0280E391E4A1E5B1EC6CE49
:1015200026EF3FEF4FEF5FEF220E331E441E551E96
:10153000BDCE10926400BACE81E080936400B6CE36
:101540008091BB009091BC0001979093BC00809368
:10155000BB00ACCE8091BB009091BC0001969093F3
:10156000BC008093BB00A2CE2091E8004091B60061
:1015700069A988A904DD9ACE5DDD98CE2091BB00D3
:101580003091BC00B501A4018AA982DC8FCE74DD44
:101590008DCE7A80882309F47DC05FA1552309F0A0
:1015A00095C09B9B93C0992784709070892B09F4F8
:1015B0008BC182EE9FEFAFEFBFEF280E391E4A1EA0
:1015C0005B1E11E01FA383CE70E09AA9923009F050
:1015D00000CF84E002CFBDA1BB2309F08FC081E41E
:1015E00099E0E5DBEAA9E23009F48FC0E33009F4C1
:1015F00045C184ED98E0DBDBFDA1FF2309F468C061
:10160000A0DB8DEE98E0D3DB6CCF84E199E0CFDBFB
:10161000A2E0EA2E05E023E0AE014F5E5F4FC50178
:10162000B4015DD2CE014196B4DB88E099E0BFDB26
:10163000B6018827992720E13EE040E050E0F4D24F
:10164000FBE09695879577956795FA95D1F7E1E058
:10165000EE2E06E021E0AE014F5E5F4F40D2CE019C
:10166000419697DB8FED73DB3CCFD501C401249607
:101670002CAD3DAD4EAD5FAD2497821B930BA40BFB
:10168000B50B52014101281639064A065B0608F0DF
:1016900054CE51CE4EA1242F332721FF0CC09B9B4B
:1016A000F0C08AE090E0A0E0B0E0280E391E4A1EAB
:1016B0005B1E91E099A724703070232B09F07FC046
:1016C00011E01EA204CE4F2D4E7F72CE11E0FFCD51
:1016D0008EE199E06CDBB2E0EB2E06E023E0AE0198
:1016E0004F5E5F4F6BA57CA58DA59EA5F8D1CE0161
:1016F00041964FDB8DEE98E05ADBF3CE8BE299E01A
:1017000056DBEAA9E23009F071CF8AED98E073CF99
:10171000A2E1B0E0EDA9FEA90F0105D3A4E1B0E07C
:10172000062CF5D284E690E009DA969881E042DA58
:1017300085B7806885BF85B78F78806285BF8895BB
:1017400089CE2091BB003091BC00B501A4018AA9CB
:101750009FDB19A6AECEA9A9A81708F0ADC0BFA5FA
:10176000BB2309F0ADC089AB89A928A9821B482FEA
:101770005527CA01880F991F840F951F9C01220FBE
:10178000331F220F331F220F331F281B390BC901B0
:10179000880F991F36FDA9C0082E892F000C881FBD
:1017A000990B000C881F991F38A9830F8093B600EE
:1017B000CA0195958795830F8093E800E4CD9B9BA4
:1017C0006EC026EF3FEF4FEF5FEF220E331E441E39
:1017D000551E11E019A71EA27ACD88E0FECD8EEF2E
:1017E00098E0E5DA2DA93EA9B90188279927EE24CA
:1017F00004E020E0AE014F5E5F4F71D1CE01419613
:10180000C8DA8AE3A4DA4AE050E0BE016F5E7F4F97
:10181000862D9927B7D139E0361508F063C0CE017F
:101820004196B7DA82EF98E0C2DA8BA99CA96CE303
:1018300070E025D2D82E8BA99CA96CE370E01FD252
:10184000772788279927EE2403E020E0AE014F5E3A
:101850005F4F45D1CE0141969CDA8AE378DA4AE0BF
:1018600050E0BE016F5E7F4F8D2D99278BD149E0EF
:101870004D15A8F5CE0141968CDA33CE80EE98E076
:10188000BACE8091BB009091BC0001969093BC00B1
:101890008093BB00A1E0A9A70ECF88AB65CF809154
:1018A000BB009091BC0001979093BC008093BB005B
:1018B00011E019A71EA20BCDF091B700FFA763CDD1
:1018C000EFA5E150EFA75FCD2EE130E040E050E022
:1018D000220E331E441E551E11E01FA3F8CC80E3D8
:1018E00036DAC8CF80E333DA9ACFCF9655CF99AFA7
:1018F00088AF52CC1F920F920FB60F9211242F93E4
:101900008F939F93EF93FF939BB12CB1E091AB002A
:10191000EF5FEF718091AC00E81749F0892F887173
:10192000E093AB00FF27E757FF4F208301C082E021
:101930008093AD00FF91EF919F918F912F910F9028
:101940000FBE0F901F9018951F920F920FB60F9217
:1019500011248F939F93EF93FF939091A90080910F
:10196000AA00981761F0E091AA00EF5FEF71E09391
:10197000AA00FF27E759FF4F80818CB901C0559815
:10198000FF91EF919F918F910F900FBE0F901F903D
:1019900018959C011092A9001092AA001092AB0019
:1019A0001092AC0097FF03C082E08BB93F77832F82
:1019B000992780BD29B988E98AB986E880BD08954C
:1019C0009091AB008091AC00981791F0E091AC0041
:1019D000EF5FEF71E093AC00FF27E757FF4F2081E7
:1019E0008091AD009927982F8827820F911D089527
:1019F00080E091E00895282F9091A9009F5F9F714A
:101A00008091AA009817E1F3E92FFF27E759FF4FCC
:101A100020839093A900559A0895CF93DF93EC010A
:101A20008881882329F02196E6DF88818823D9F7E9
:101A3000DF91CF910895CF93DF93FC0184918823A8
:101A400049F0EF012196D7DFFE012196E4918E2F18
:101A5000EE23C9F7DF91CF910895662339F0FC0199
:101A600080816193682F8823D9F701C0FC0110821F
:101A70000895FF920F931F93CF93DF93EA01F22E05
:101A8000022F0F5F2AE030E09CD0FE010190002081
:101A9000E9F731971E2F1C1B101730F460E3CE01BD
:101AA000DCDF1F5F1017D0F3FE01319680818823A1
:101AB000E1F79F01002359F09F2D01C080818183B0
:101AC00031979150D8F7F901EF19F10931978EE26A
:101AD0008183DF91CF911F910F91FF900895EF9235
:101AE0000F931F93CF93DF93EA01122FC2DFFE0102
:101AF00001900020E9F731974E2F4C1B212F2E1912
:101B0000EE2009F42F5F121654F5E42FFF27822FE1
:101B1000992787FD9095E81BF90BEC0FFD1F1082AC
:101B2000421B041B101644F5242F2F5F802F99278A
:101B300087FD9095FE01E40FF11DE80FF91FDF010D
:101B4000A81BB90B8C9180833197215011971216E5
:101B5000CCF380E2808331970150E1F70DC01E1570
:101B600000F7FE01E40FF11DE11A8E2D90E3919331
:101B70008150E8F74E0DD5CFDF91CF911F910F9196
:101B8000EF900895FB019F01E8944230BCF045328C
:101B9000ACF44A3029F497FB1EF4909581959F4F41
:101BA000642F77276CD0805D8A330CF0895D819338
:101BB000CB010097A9F716F45DE251931082C90199
:101BC00023C0FA01CF93FF93EF932230C4F0253264
:101BD000B4F4C22F2C2F332744275527FF93EF93BC
:101BE00062D0EF91FF91605D6A330CF0695D6193A3
:101BF000B901CA01605070408040904059F710828E
:101C00008F919F91CF9100C0DC01FC01672F7191F2
:101C10007723E1F7329704C07C916D9370836291D2
:101C2000AE17BF07C8F30895629FD001739FF001FC
:101C3000829FE00DF11D649FE00DF11D929FF00D5C
:101C4000839FF00D749FF00D659FF00D9927729F93
:101C5000B00DE11DF91F639FB00DE11DF91FBD011E
:101C6000CF0111240895991B79E004C0991F96179C
:101C700008F0961B881F7A95C9F780950895AA1BCE
:101C8000BB1B51E107C0AA1FBB1FA617B70710F067
:101C9000A61BB70B881F991F5A95A9F78095909599
:101CA000BC01CD010895A1E21A2EAA1BBB1BFD01A8
:101CB0000DC0AA1FBB1FEE1FFF1FA217B307E4072B
:101CC000F50720F0A21BB30BE40BF50B661F771F83
:101CD000881F991F1A9469F7609570958095909563
:101CE0009B01AC01BD01CF010895E199FECFBFBBBF
:101CF000AEBBE09A11960DB20895F7DF01921A94E7
:101D0000E1F70895F2DFE02DF0DFF02D0895E1997D
:101D1000FECFBFBBAEBB0DBA11960FB6F894E29AD8
:101D2000E19A0FBE0895F3DF012CF1DF112408952D
:101D30000190EDDF1A94E1F70895FFCFEA6D0000FE
:101D4000010000919F918F910F900FBE0F901F90F7
:101D500018959C011092A9001092AA001092AB0055
:101D60001092AC0097FF03C082E08BB93F77832FBE
:101D7000992780BD29B988E98AB986E880BD089588
:101D80009091AB008091AC00981791F0E091AC007D
:101D9000EF5FEF71E093AC00FF27E757FF4F208123
:101DA0008091AD009927982F8827820F911D089563
:101DB00080E091E00895282F9091A9009F5F9F7186
:101DC0008091AA009817E1F3E92FFF27E759FF4F09
:101DD00020839093A900559A0895CF93DF93EC0147
:101DE0008881882329F02196E6DF88818823D9F726
:101DF000DF91CF910895CF93DF93FC0184918823E5
:101E0000F8940FE50DBF04E00EBF22243324909A0E
:101E1000919A899A41E050EA0CE0F101EF01F10159
:101E2000019700408099E1F781F12197349668F19C
:101E3000809BFBCF0F2EC5950694E9F72397269636
:101E400068F7EA35F20550F3F797F695E7952F0115
:101E5000CAE0E6EBFFE10590002031F078D00016F3
:101E6000D1F3CA9591F0F5CF06EA8AD070D0E1F7A8
:101E70000AEA86D06CD0F1F76AD0F1F3F101E89468
:101E80000430F0F059F1063018F422BA21BAB8C083
:101E900031F45DD05CD0672859F331010FC00730B1
:101EA00059F455D019F453D0005821F00590001280
:101EB0006894F7CF1EF0DCCF07EADBCF0BEAD9CF6F
:101EC000ECEBFFE1C0E0EC0FF21DC4910150D8F73C
:101ED00008EA56D00591C150E0F7CACFA0E6B0E0BD
:101EE000ED0135D021F433D00058689431F0E894F6
:101EF0000D93A03204E0B007A1F7AC17BD0731F194
:101F0000A0E2B4E0E054FC4F10E232971E900E9035
:101F100001E015D01A95C9F7E0301EE1F107A8F4E9
:101F200003E00DD005E009D0AC17BD0769F776F0E6
:101F3000E054FC4F09EA24D0D4CF01D001E107BF1F
:101F4000E89507B700FDFDCF0895B8CF91CF809BEE
:101F5000FECF8099FECF18E0C2019695879523D0D9
:101F600021D006958099006807FD642676946794D1
:101F700008F4642608F475261A9591F7053A089531
:101F800011D09198149119E0009500C000C00AD0BA
:101F9000069518F40000919802C0919A00C01A9515
:101FA000A1F70895C2010497F0F78D3F18F011F0E2
:101FB0008F3F01F00895506564610000030107033D
:101FC00003C0041E930704001E00FFFFFFFFFFFF76
:1020000050C300000002AC070100000208C9010033
:102010000002000000000032000000070100FF1075
:10202000020202FFFFFFFFFFFFFFFFFFFFFFFFFFB7
:10214000FFFFFFFFFFFFFFFFFFFFFFFF213D47AF47
:00000001FF
